:100000000C946B000C9416070C9443070C9493000B
:100010000C9493000C9493000C9493000C94930014
:100020000C9493000C9493000C9493000C94510541
:100030000C9493000C9493000C9493000C949300F4
:100040000C9470070C9493000C9450090C949E0926
:100050000C9493000C9493000C9493000C949300D4
:100060000C9493000C9493000000010008004000E1
:1000700000010004050D00000000240027002A00F4
:1000800000000000250028002B00000000002300D5
:1000900026002900040404040404040402020202E9
:1000A000020203030303030301020408102040803B
:1000B00001020408102001020408102000000007BB
:1000C0000002010000030406000000000000000020
:1000D000A7005102830A11241FBECFEFD8E0DEBF74
:1000E000CDBF11E0A0E0B1E0ECE7F6E102C0059081
:1000F0000D92A03BB107D9F713E0A0EBB1E001C02E
:100100001D92AD36B107E1F710E0C6EDD0E004C0B6
:100110002297FE010E94380BC03DD107C9F70E940B
:10012000D90A0C943C0B0C940000FB01DC0102C0CA
:1001300005900D9241505040D8F70895FB01DC0125
:1001400002C001900D9241505040D8F70895EF92AF
:100150000F9380EB91E060ED77E04BE02CE00AE05C
:10016000EE240E9495060F91EF9008951F9382E070
:100170000E94FC08182F6AE070E080E090E00E9486
:100180000108113029F4609104017091050104C047
:100190006091060170910701DB010D900020E9F7E5
:1001A0001197A61BB70B80EB91E04A2F0E94C40267
:1001B00080EB91E00E944A0162E370E080E090E011
:1001C0000E9401081F9108958DE061E00E94690876
:1001D00082E062E00E94690814C08DE061E00E9444
:1001E000A80864E670E080E090E00E9401088DE0DD
:1001F00060E00E94A80864E670E080E090E00E9461
:10020000010880EB91E00E947406882331F3089581
:100210006827462F4295407F462750E0742F662777
:10022000292F30E0622B732BCA01A3E0880F991F9E
:10023000AA95E1F768277927F4E056954795FA954E
:10024000E1F764277527CB010895FC018CE091E06C
:1002500091838083138212828FEF848382878387C6
:1002600014861586108A1786128A118A148A138AB0
:10027000089581E00895CF93DF93EC01E881F9813F
:100280000280F381E02DCE0109958823B9F3DF9137
:10029000CF910895FC01828193810397E1F381E07E
:1002A0000895FC0165830895FC0164830895FC01B1
:1002B00062870895FC0163870895FC0164870895AF
:1002C000FC01409585854823462B45870895FC0110
:1002D00086810895FC0187810895FC018085089539
:1002E000FC018185089580E00895AF92BF92CF927E
:1002F000DF92EF92FF920F931F93CF93DF93EC0166
:100300008B010E94B8075B016C01780100E010E0EE
:1003100006C08A819B81039711F081E00CC00E9486
:10032000B8076A197B098C099D096E157F0580073E
:10033000910778F380E0DF91CF911F910F91FF90AB
:10034000EF90DF90CF90BF90AF900895AF92BF92A3
:10035000CF92DF92EF92FF920F931F93CF93DF9391
:10036000EC018B010E94B8075B016C01780100E091
:1003700010E00BC0E881F9810280F381E02DCE010D
:100380000995882311F081E00CC00E94B8076A1912
:100390007B098C099D096E157F058007910750F335
:1003A00080E0DF91CF911F910F91FF90EF90DF9050
:1003B000CF90BF90AF90089508950895FC0188E311
:1003C00091E0918380837383628355834483378371
:1003D00026830895FC01758364830895FC01778367
:1003E00066830895FC017383628308956EBD0DB426
:1003F00007FEFDCF8EB508958CB580688CBD08953D
:100400008CB58F778CBD08950E94DC060895CF933C
:10041000DF93EC018E819F81009771F0813091050F
:1004200011F484E00AC08230910511F488E005C01F
:10043000039711F48CE001C080E00E94E90620E0FF
:100440008C819D81019709F021E0822F0E94E006B6
:100450008A819B818230910569F0833091051CF47B
:10046000019731F403C005971CF406C085E005C070
:1004700081E003C080E001C084E00E94EE060E949B
:10048000FF06DF91CF9108950F931F938C010E9477
:10049000DE018CE491E0F801918380831F910F913C
:1004A00008958CEA92E060E070E040E050E020E0E7
:1004B00030E00E94440208958CE30895EF92FF9289
:1004C0001F93CF93DF93EC012FEF3FEF10E089E60E
:1004D000E82EF12CEC0EFD1E09C0FE01E10FF11D0E
:1004E000C90165A10E9408019C011F5FF70180817D
:1004F000181798F3285B304F39F08F85988901964B
:10050000988B8F871D8E19C08EA18E838FA18F83AC
:1005100088A5888789A589878D81882339F49E815C
:100520008C81981719F08E818F3F39F489899A89C7
:1005300001969A8B898B81E08D8FDF91CF911F91EE
:10054000FF90EF900895FC01862F638D6827818DC1
:100550000E94A8080895CF93DF93EC018A819B81C4
:10056000039779F0C659DF4F199219921882CC5629
:10057000D040CE0161E00E94A30283E090E09B8323
:100580008A83DF91CF9108959F92AF92BF92CF92CD
:10059000DF92EF92FF920F931F93CF93DF93EC01C3
:1005A000A62E972EB42E8CE3841710F480E001C1A0
:1005B00035E7E32EF12CEC0EFD1E042F095FE881D8
:1005C000F9810484F585E02DCE0109958FEF9FEF29
:1005D000602F0E94080110E0F80124E0F595E795EE
:1005E0002A95E1F7E857FE4F2081F70120830F702D
:1005F000107008571E4FF8012081F70121836A858A
:100600000E940801EA85F0E0B4E0F595E795BA9517
:10061000E1F7E857FE4F2081F7012283EA85F0E0F9
:10062000EF70F070E857FE4F2081F70123836B8550
:100630000E940801EB85F0E0A4E0F595E795AA9506
:10064000E1F7E857FE4F2081F7012483EB85F0E0C6
:10065000EF70F070E857FE4F2081F70125836C851D
:100660000E940801EC85F0E074E0F595E7957A9535
:10067000E1F7E857FE4F2081F7012683EC85F0E093
:10068000EF70F070E857FE4F2081F70127836D85EA
:100690000E940801DC01ED85F0E064E0F595E79546
:1006A0006A95E1F7E857FE4F8081F7018087ED8575
:1006B000F0E0EF70F070E857FE4F8081F70181871E
:1006C00067012A2D392DC9018C0120C0CD01F80107
:1006D00060810E940801DC01F8018081E82FF0E0D0
:1006E00054E0F595E7955A95E1F7E857FE4F80817C
:1006F000F6018087F80181918F01E82FF0E0EF701B
:10070000F070E857FE4F8081F601818782E090E02B
:10071000C80ED91E802F8A198B15C0F28B2D90E040
:100720000596880F991FA095B095A701480F591FEE
:10073000FD0134E0F695E7953A95E1F7EF70F0703A
:10074000E857FE4F2081FA0120830196A701480F48
:10075000591FFD01EF70F070E857FE4F2081FA013C
:1007600020830196A701480F591FFD01EF2FFF2796
:10077000E295EF70E857FE4F2081FA012083019641
:10078000E80EF91EAB2FBB27AF70B070A857BE4F55
:100790002C91F7012083C550DF4F875F8883CB5FA3
:1007A000D040CE010E94AB02D093B502C093B402F8
:1007B00081E0DF91CF911F910F91FF90EF90DF903B
:1007C000CF90BF90AF909F900895CF93DF93EC01AF
:1007D0008A819B81049761F0CE0160E00E94A302B0
:1007E000888D60E00E94A80884E090E09B838A8363
:1007F000DF91CF910895CF93DF93EC018A819B81A4
:10080000039711F480E00BC0CE010E94E5038C8DAC
:10081000882321F0CE010E945E021C8E8D8DDF9117
:10082000CF910895CF93DF93EC018A819B8102974A
:1008300061F0CE0160E00E94A302888D60E00E941A
:10084000A80882E090E09B838A83DF91CF9108958E
:10085000EF92FF920F931F93CF93DF93EC01FC0174
:10086000E459FF4F80818F5F80838150D1F54AE644
:10087000E42EF12CEC0EFD1EF7019081C550DF4FE8
:100880008881CB5FD040981748F0CE010E941204B7
:100890008B899C8901969C8B8B8B23C08E0105597B
:1008A0001F4FF8018081FE01E90FF11DE359FF4F51
:1008B000608170E0082E02C0759567950A94E2F792
:1008C000617070708F5FF8018083888D0E94A80826
:1008D000F8018081863028F01082F70180818F5FD7
:1008E0008083FE01E459FF4F8081883008F0108238
:1008F000DF91CF911F910F91FF90EF900895CF93CB
:10090000DF93EC018F890E94FC0830E020E0892B06
:1009100009F021E08A8D281331E0832FDF91CF91F8
:100920000895CF93DF93EC010E947F04982F8823D2
:1009300019F08F8D8F5F8F8F8E8D981759F028A1AA
:1009400088A1803510F08DE101C08BE0820F88A373
:100950009E8F03C088A18C5E88A388A1803A08F48A
:100960008CC08AA19BA1969587959BA38AA38F8D06
:10097000853028F08AA19BA198609BA38AA388A1B7
:10098000805A88A31F8E89A1882309F46BC08CA18B
:100990008F5F8CA38CA18C3008F46FC08AA19BA1BF
:1009A000282F2F73322F36953695387098E008C06F
:1009B000E32FF0E0E857FE4F8081281721F03F5FDA
:1009C0009150B0F730E08AA19BA156E096958795AB
:1009D0005A95E1F7982F282F26952695287048E0FC
:1009E00008C0E22FF0E0E857FE4F8081981721F011
:1009F0002F5F4150B0F720E0932F9295907F922B7C
:100A0000C759DF4F8881C956D040882389F4FE0139
:100A1000E859FF4F90838081873018F080818434BB
:100A200038F019A28F8598890196988B8F8725C0F9
:100A3000DE01A759BF4F8C91FE01E80FF11D95A370
:100A40008F5F8C939C91C859DF4F8881C856D040E6
:100A5000981730F019A281E08C8FCE010E94120409
:100A60001CA20BC08AA19BA188539B4031F481E05A
:100A700089A31CA2C759DF4F1882DF91CF91089537
:100A8000FC0182819381049721F4CF010E9491049B
:100A9000089582819381039719F4CF010E9428045D
:100AA00008951F920F920FB60F9211242F933F9328
:100AB0004F935F936F937F938F939F93AF93BF9366
:100AC000EF93FF938091B4029091B5020E9440058C
:100AD000FF91EF91BF91AF919F918F917F916F9116
:100AE0005F914F913F912F910F900FBE0F901F90EC
:100AF0001895EF92FF920F931F93CF93DF93EC0122
:100B00007B018A01E881F9810280F381E02D09955A
:100B10008823E9F0E114F104C1F001151105A9F0F1
:100B2000C759DF4F9881C956D0409750F80180814E
:100B3000981708F49083F80140819E01265D3F4F8D
:100B4000C701B90150E00E949E001D8E81E0DF9137
:100B5000CF911F910F91FF90EF9008952F923F92A8
:100B60005F926F927F928F929F92AF92BF92CF923D
:100B7000DF92EF92FF920F931F93DF93CF9300D0FA
:100B800000D000D0CDB7DEB71A013901611571056B
:100B900021F4D9011D921C925DC05B01CC24DD249F
:100BA000A3E0AA0CBB1CCC1CDD1CAA95D1F7F1E07C
:100BB0008F2E912CCA01A0E0B0E08B839C83AD8383
:100BC000BE83582CB401660F771F68597F4FCE0142
:100BD000019642E050E00E94950029813A8140E070
:100BE00050E060E074E284EF90E00E94140BCA01D0
:100BF000B901A60195010E94140B79018A0192E0C6
:100C0000E916F1040105110548F08B819C81AD8145
:100C1000BE81E816F9060A071B0740F053940894B2
:100C2000811C911C97E08916910459F6A6E05A168A
:100C300071F0B2E0EB16F1040105110540F0C101BD
:100C4000A0E0B0E08E159F05A007B10728F4F301DE
:100C500011821082552403C0D301ED92FC92852DA0
:100C600026960FB6F894DEBF0FBECDBFCF91DF91B1
:100C70001F910F91FF90EF90DF90CF90BF90AF90BA
:100C80009F908F907F906F905F903F902F900895EE
:100C9000DF93CF9300D0CDB7DEB7FC0165897689AD
:100CA0004FEF5FEF9E012F5F3F4F0E94AE05982FE1
:100CB0008823A9F01092800088E0809381008091C1
:100CC0008100892B8093810089819A81909389008A
:100CD0008093880080916F00826080936F000F90F6
:100CE0000F90CF91DF910895CF93DF93EC010E9495
:100CF00039018823B9F0D093B502C093B402888D2E
:100D000061E00E9469088F8960E00E946908898D0E
:100D100061E00E946908CE010E941204CE010E9487
:100D2000480681E0DF91CF910895AF92BF92CF92B4
:100D3000DF92EF92FF920F931F93DF93CF93CDB784
:100D4000DEB728970FB6F894DEBF0FBECDBF5C01AB
:100D50006B01142FF22E0E94250180E691E0F5012F
:100D600091838083D68AC58A178BF08E018FE38E9C
:100D7000DE011196E8E9F1E088E001900D928150E2
:100D8000E1F7D501A359BF4FFE01319688E00190EC
:100D90000D928150E1F728960FB6F894DEBF0FBE92
:100DA000CDBFCF91DF911F910F91FF90EF90DF901A
:100DB000CF90BF90AF9008958CB58F7B8CBD089578
:100DC000882319F48CB5806202C08CB58F7D8CBDF0
:100DD00008959CB5937F982B9CBD08952CB5382F12
:100DE00033702C7F322B3CBD2DB590E095958795C7
:100DF0009595879581702E7F822B8DBD08958AE011
:100E000061E00E94A8088AE061E00E9469088CB550
:100E100080618CBD8CB580648CBD8DE061E00E94EA
:100E200069088BE061E00E94690808951F920F92A3
:100E30000FB60F9211242F933F934F935F936F93AD
:100E40007F938F939F93AF93BF93EF93FF93809183
:100E5000B6029091B702892B29F0E091B602F09189
:100E6000B7020995FF91EF91BF91AF919F918F913B
:100E70007F916F915F914F913F912F910F900FBE96
:100E80000F901F9018951F920F920FB60F9211247A
:100E90002F933F934F935F936F937F938F939F9382
:100EA000AF93BF93EF93FF938091B8029091B902F3
:100EB000892B29F0E091B802F091B9020995FF91D0
:100EC000EF91BF91AF919F918F917F916F915F91C2
:100ED0004F913F912F910F900FBE0F901F9018953B
:100EE0001F920F920FB60F9211242F933F938F935F
:100EF0009F93AF93BF938091BE029091BF02A09148
:100F0000C002B091C1023091C2020196A11DB11D73
:100F1000232F2D5F2D3720F02D570196A11DB11DD8
:100F20002093C2028093BE029093BF02A093C0029E
:100F3000B093C1028091BA029091BB02A091BC0211
:100F4000B091BD020196A11DB11D8093BA0290938C
:100F5000BB02A093BC02B093BD02BF91AF919F9121
:100F60008F913F912F910F900FBE0F901F9018956A
:100F70008FB7F8942091BE023091BF024091C00219
:100F80005091C1028FBFB901CA010895789484B508
:100F9000826084BD84B5816084BD85B5826085BD75
:100FA00085B5816085BDEEE6F0E08081816080835B
:100FB000E1E8F0E01082808182608083808181603E
:100FC0008083E0E8F0E0808181608083E1EBF0E005
:100FD000808184608083E0EBF0E0808181608083A9
:100FE000EAE7F0E080818460808380818260808392
:100FF0008081816080838081806880831092C100BD
:101000000895EF92FF920F931F93CF93DF937B018D
:101010008C013FB7F8948091BA029091BB02A091E5
:10102000BC02B091BD0226B5A89B05C02F3F19F0A8
:101030000196A11DB11D3FBFBA2FA92F982F882758
:10104000820F911DA11DB11D52E0880F991FAA1F8B
:10105000BB1F5A95D1F7EC0130C00E94130B3FB76C
:10106000F8948091BA029091BB02A091BC02B09119
:10107000BD0226B5A89B05C02F3F19F00196A11D02
:10108000B11D3FBFBA2FA92F982F8827820F911D1E
:10109000A11DB11D32E0880F991FAA1FBB1F3A95F1
:1010A000D1F78C1B9D0B885E9340B8F20894E10841
:1010B000F10801091109C851DC4FE114F1040105DF
:1010C000110559F6DF91CF911F910F91FF90EF908D
:1010D0000895CF93DF93482F50E0CA0188559F4F62
:1010E000FC0134914C565F4FFA018491882369F1D9
:1010F00090E0880F991FFC01EA58FF4FA591B49129
:10110000FC01E058FF4FC591D491662351F42FB7ED
:10111000F8948C91932F909589238C9388818923BF
:101120000BC0623061F42FB7F8948C91932F909597
:1011300089238C938881832B88832FBF06C09FB718
:10114000F8948C91832B8C939FBFDF91CF9108955E
:10115000482F50E0CA0184549F4FFC012491CA01DA
:1011600088559F4FFC0194914C565F4FFA01349182
:10117000332309F440C0222351F1233071F024308D
:1011800028F42130A1F0223011F514C02630B1F03E
:101190002730C1F02430D9F404C0809180008F77CB
:1011A00003C0809180008F7D8093800010C084B543
:1011B0008F7702C084B58F7D84BD09C08091B00057
:1011C0008F7703C08091B0008F7D8093B000E32FB4
:1011D000F0E0EE0FFF1FE058FF4FA591B4912FB73D
:1011E000F894662321F48C919095892302C08C9108
:1011F000892B8C932FBF0895682F70E0CB01845406
:101200009F4FFC012491CB0188559F4FFC014491D5
:101210006C567F4FFB019491992319F420E030E044
:101220003CC0222351F1233071F0243028F42130C6
:10123000A1F0223011F514C02630B1F02730C1F0F2
:101240002430D9F404C0809180008F7703C080914E
:1012500080008F7D8093800010C084B58F7702C09E
:1012600084B58F7D84BD09C08091B0008F7703C0A5
:101270008091B0008F7D8093B000892F90E0880F1F
:10128000991F86579F4FFC01A591B4918C9120E046
:1012900030E0842311F021E030E0C9010895089581
:1012A0001F920F920FB60F9211242F933F934F93DB
:1012B0008F939F93EF93FF938091C00082FD1DC099
:1012C0004091C60020910303309104032F5F3F4FEC
:1012D0002F7330708091050390910603281739070A
:1012E00071F0E0910303F0910403ED53FD4F40834F
:1012F000309304032093030302C08091C600FF9142
:10130000EF919F918F914F913F912F910F900FBE31
:101310000F901F901895E0915703F0915803E05CEF
:10132000FF4F8191919120813181821B930B8F73AB
:101330009070892B11F00E944F0908951F920F920F
:101340000FB60F9211242F933F938F939F93EF9398
:10135000FF93209147033091480380914903909176
:101360004A032817390731F48091C1008F7D80939B
:10137000C10014C0E0914903F0914A03E95FFC4FBA
:1013800020818091490390914A0301968F73907058
:1013900090934A03809349032093C600FF91EF91F5
:1013A0009F918F913F912F910F900FBE0F901F90A3
:1013B0001895DC011C96ED91FC911D97E05CFF4FA8
:1013C0002191319180819181281B390B2F733070CD
:1013D000C9010895DC011C96ED91FC911D97E05C1C
:1013E000FF4F20813181E054F040DF01AE5BBF4F01
:1013F0008D919C9111972817390719F42FEF3FEF22
:1014000007C08D919C91E80FF91F8081282F30E053
:10141000C9010895DC011C96ED91FC911D97E05CDB
:10142000FF4F20813181E054F040DF01AE5BBF4FC0
:101430008D919C9111972817390719F42FEF3FEFE1
:1014400010C08D919C911197E80FF91F20818D910B
:101450009C91119701968F73907011969C938E9327
:1014600030E0C9010895DC0191968C919197882311
:1014700039F05496ED91FC915597808186FFF9CF14
:1014800091961C920895CF93DF93EC01EE85FF8532
:10149000E05CFF4F20813181E054F0402F5F3F4FEF
:1014A0002F733070DF01AE5BBF4F8D919C91119710
:1014B00028173907D1F3E05CFF4F80819181E05418
:1014C000F040E80FF91F6083EE85FF85E05CFF4F79
:1014D00031832083EE89FF89208181E090E00F8CA9
:1014E00002C0880F991F0A94E2F7282B208381E01D
:1014F00089A3EC89FD8980818064808381E090E00C
:10150000DF91CF91089510924E0310924D0388EE13
:1015100093E0A0E0B0E080934F0390935003A0933A
:101520005103B093520384EA91E090934C0380936B
:101530004B0383EC92E0909358038093570387E02A
:1015400093E090935A038093590385EC90E0909335
:101550005C0380935B0384EC90E090935E03809344
:101560005D0380EC90E09093600380935F0381ECD7
:1015700090E0909362038093610382EC90E09093FB
:1015800064038093630386EC90E0909366038093FA
:10159000650384E08093670383E08093680387E0BA
:1015A0008093690385E080936A0381E080936B03F5
:1015B0000895CF93DF930E94C6070E94E400CBE812
:1015C000D9E00E94B6002097E1F30E948B09F9CF81
:1015D0000895CF92DF92EF92FF920F931F93CF93D4
:1015E000DF937C016B018A01C0E0D0E00FC0D6011F
:1015F0006D916D01D701ED91FC910190F081E02D8D
:10160000C7010995C80FD91F0150104001151105D8
:1016100071F7CE01DF91CF911F910F91FF90EF9065
:10162000DF90CF9008950895A1E21A2EAA1BBB1B4C
:10163000FD010DC0AA1FBB1FEE1FFF1FA217B3079E
:10164000E407F50720F0A21BB30BE40BF50B661FB4
:10165000771F881F991F1A9469F760957095809578
:1016600090959B01AC01BD01CF010895EE0FFF1FC6
:0C1670000590F491E02D0994F894FFCF50
:10167C003100300000010201000000003901E80ACD
:10168C00E80AE80AE80A3B014A017501A60154017F
:10169C0057015A015D016001510167016A016D0139
:1016AC007001730100000000E80ADC01DD01E80AAA
:1016BC00E80AEA01EE01F20100000000F601FC016B
:1016CC00000207020402EA01EE01F2010000000030
:1016DC007406FB037905C4025C023B014A017501E7
:1016EC00A601540157015A015D01600151016701C6
:1016FC006A016D01700173010D0E131516191A1C78
:10170C00232526292A2C32342A2A2A2A2A2A382C1A
:10171C0000000000430AE90AD9090A0AEA09330A57
:00000001FF
